:104760000000090101240200000301FA0400FA0517
:1047700000020A0A5A0B000F0C00FA0D00030E008B
:10478000030F0132100096120132130AFA140102CB
:1047900015000217010A18010A1905321A010A1B2D
:1047A000010A1C053223011E2400642A00FA2B0092
:1047B000FA2C50782D003C2E00462F001E3000644D
:1047C0003250783300003432FA35016436016437F0
:1047D0000150380A643C00643E003C3F000140FF49
:1047E000FF411450420A5A430AC844053245007832
:1047F0004600FA4701234802034C00FA4EFFFF50DF
:104800000404510596521432530B28540A9656014B
:1048100002570546580002590A465A32FA5B010A05
:104820005C14325E000A5F00FE61FFFF64021167E4
:1048300001036A0A3C6B00006C3296780132790100
:1048400032FAFAFA0000090101240200000301FA19
:104850000400FA0500020A0A5A0B000F0C00FA0DB8
:1048600000030E00030F0132100096120132130AEA
:10487000FA14010215000017010A18010A1905327D
:104880001A010A1B010A1C053223011E2400642A96
:1048900000FA2B00FA2C50782D003C2E00462F00F9
:1048A0001E3000643250783300003432FA3501642F
:1048B000360164370150380A643C00643E003C3FD6
:1048C000000140FFFF411450420A5A430AC8440500
:1048D000324500784600FA4701234802024C00FAAC
:1048E0004EFFFF500404510596521432530B2854C6
:1048F0000A96560101570546580001590A465A3290
:10490000FA5B010A5C14325E000A5F00FE61FFFF81
:104910006402116701036A0A3C6B00006C329678EE
:104920000132790132FAFAFA0065006F00790083EA
:10493000008D009700A100AC00B600C000CA00D4F2
:1049400000DE00E800F2005B0063006A0072007A9B
:10495000008200890091009900A100A800B000B871
:1049600000BF00C700CF00D600DF00E600EE00F673
:1049700000400046004C00520059005F0065006B8B
:1049800000710077007D00830089008F0095009CF6
:1049900000A200A800AE00B400BA00C000C600CC5F
:0C49A00000D200D900DF00E500EB00F1C0
:10009E0085F95085FA517E017F00E551124C36E507
:1000AE00502FFF50010E8E338F34900014E0FCA3BE
:1000BE00E0FDEF2DFDEE3CFC8C358D362275A71044
:1000CE0085F95085FA517E017F00E551124C36E5D7
:1000DE00502FFF50010E8E338F349000CBE0B402C0
:1000EE0010AC56AD57EF2DFDEE3CFC8C358D3680A9
:1000FE0016AE33AF34900014E0FCA3E0FDEF2DFDFF
:10010E00EE3CFC8C358D3622AE33AF34740A8E0441
:10011E008F05FF124C188C358D36AE33AF34740A02
:10012E008E048F05FF124C518C338D34E5344533DC
:10013E006013740AC39534FFE49533FE8E338F3407
:10014E007835124C93E550A835B80015D395364046
:10015E0010E550C39536FFE49535FE8E358F36800B
:10016E0010E5502424C39536FFE49535FE8E358F69
:10017E0036AE35AF3674246F4E700B75362375352B
:10018E0000755001800375500022900079E0B40193
:10019E0004C20B8002D20B90007AE0B40104C20CB0
:1001AE008002D20C9000B7E075F0DCA4FFAEF074C4
:1001BE000A8E048F05FF124C1890079FECF0A3EDEA
:1001CE00F0A208401674038C068D07124C3674018B
:1001DE00124C2890079DEEF0A3EFF07E017F009069
:1001EE000075E0124C369000B8E08E048F05FF12B9
:1001FE004C18740AFF124C188D399000C1E075F03E
:10020E00DCA4FFAEF0740A8E048F05FF124C18901A
:10021E0007A3ECF0A3EDF09000C3E060139000C3D1
:10022E00E0F5F0741684FF7E00EF9007ABF08006C9
:10023E0074649007ABF09000A2E0B40B0874E390E6
:10024E000064F080499000A2E0B419129000B8E06A
:10025E0090491312008CE493900064F0803090006B
:10026E00A2E0B41E129000B8E090493112008CE466
:10027E0093900064F080179000A2E0B428109000D4
:10028E00B8E090495B12008CE493900064F090000B
:10029E0040E0C39405502274019000BBF09000BD65
:1002AE00E0B4020674019000BDF09000ADE0D3946E
:1002BE0002400674029000ADF09000D5E0B4011734
:1002CE00900020740FF0A374FFF0900022E4F0A3CE
:1002DE00F074029000D5F09000D5E0B40341900088
:1002EE0022E0FEA3E0FF900020E0FCA3E0FD124C14
:1002FE008B7410124C367408124C28EF900061F07B
:10030E00EF700674FF900061F074009000D5F090CD
:10031E000021E0900062F0900020E0900063F090E9
:10032E000066E090002CF090002CE0D39412400D6B
:10033E0090002CE0C3941290002DF0800A90002CB7
:10034E00E0241290002DF090002CE0B4240E9000CA
:10035E002C7401F09000307401F08005900030E4B0
:10036E00F090002DE0B4240E90002D7401F090005A
:10037E00317401F08005900031E4F0900066E0FEEB
:10038E009000C9E02E900033F0900033E0D3942417
:10039E00400B900033E0C39424900033F090003370
:1003AE00E0B412067413900033F0900033E0B424DE
:1003BE00069000337401F0900033E0D39412400D98
:1003CE00900033E0C39412900034F0800A90003312
:1003DE00E02412900034F09000ACE090002EF090EB
:1003EE00002EE0B41206741390002EF090002EE052
:1003FE00D39412400D90002EE0C3941290002FF073
:10040E00800A90002EE0241290002FF022C293C298
:10041E0094C291C292C287C290E5B554EFF5B5E58C
:10042E00B554DFF5B5C296C295C2A0C297C2A2C29C
:10043E00A1E5B554BFF5B5E5B5547FF5B5E5B554B1
:10044E00FBF5B5C20D7537469000AFE070057549E6
:10045E0002800375490390000874FFF0A374DCF06A
:10046E00900090E090000EF8E4F0E8A3F0C212C203
:10047E001474C8900024F074C8900028F0752600FB
:10048E00752500C208756C00E54BB40903754B0069
:10049E00753C00900016E4F0A3F0754C1E75280014
:1004AE00752700C210C21190079FE0FEA3E0FF74F3
:1004BE0003124C367401124C2890079DEEF0A3EFF8
:1004CE00F0C20390000CE4F0A3F0C21F2285F95095
:1004DE0085FA517E017F00E551124C36E5502FFF13
:1004EE0050010E8E338F3490079FE0FCA3E0FDEF9A
:1004FE002DFDEE3CFC8C358D36E536F5FDE535F5FE
:10050E00FE22053D229000ADE0B403539000CBE0F7
:10051E00B4012EA2D8B34004C293C287A2D9B3406D
:10052E0004C294C290A2DAB34008C291E5B554EF6A
:10053E00F5B5A2DBB34008C292E5B554DFF5B58040
:10054E001CA2D8B34002C293A2D9B34002C294A255
:10055E00DAB34002C291A2DBB34002C2928012A271
:10056E00D8B34004C293C287A2D9B34004C294C286
:10057E0090A2DCB34004C296C29575D8402285A7DE
:10058E004F75A710A2D8B34002C287A2D9B34002BA
:10059E00C290A2DAB34006E5B554EFF5B5A2DBB3CF
:1005AE004006E5B554DFF5B575D840854FA72290C6
:1005BE000047E4936406600280FE74C89007A5F8B5
:1005CE00E4F0E8A3F075B50075840175A70075FF1A
:1005DE008075EF06900032E4F075C91075A70F759F
:1005EE00A1C775A70075D90075CE0C75A70F75F14B
:1005FE00FE75F2FF75F30775F47875A4BA75A5FF4D
:10060E0075A60775AE0075AFFF75D48175D5FF75EC
:10061E00D6FF75D7FF75A70075A20175A14775F8AE
:10062E000975D80075D90475DA0975DB0975DC0909
:10063E0075DD0975DE0975D84075A71075D800757A
:10064E00D90475DA0975DB0975DC0975DD0975D80C
:10065E004075A70075E60875E71075BC0175BE04F8
:10066E0075BD6C75BE0775BDA075BE0875BD0175EF
:10067E00BC0075BB1875BC2075BA0875E88075D1BD
:10068E001375A70F75E10575E20075C740C293C2D9
:10069E0094C291C292C287C290E5B554EFF5B5E50A
:1006AE00B554DFF5B5C296C295C2A0C297C2A2C21A
:1006BE00A1E5B554BFF5B5E5B5547FF5B5E5B5542F
:1006CE00FBF5B5759700759780740A124C087597EF
:1006DE00C0E5975420700280F8758F0275A700D27E
:1006EE00AF75980075A90C75A70F75AB4375ADFB6B
:1006FE0075AC1E75A71075C91875CA0075CB007537
:10070E00C80475A700758912758E04758C00758ADC
:10071E0000C2A9D28C758D00758B00D2ABD28E75AE
:10072E00D944753200753100752E00752D00754651
:10073E0000754700C29974C8F509750800122BA6FA
:10074E0075B50074639007A5F8E4F0E8A3F0122ED7
:10075E00327464F509750800122BA6C21B90004F67
:10076E00E0B40108A2B54002D21B802E90004FE0EB
:10077E00B4021175A70F75F30F75A700A2A340025F
:10078E00D21B801690004FE0B4030F75A70F75F3C0
:10079E001775A700A2A44002D21BA21BB3500302DE
:1007AE00089674089007A5F8E4F0E8A3F0122D015E
:1007BE007464F509750800122BA674099007A5F844
:1007CE00E4F0E8A3F0122D017464F5097508001227
:1007DE002BA6740A9007A5F8E4F0E8A3F0122D01F9
:1007EE007464F509750800122BA6740B9007A5F812
:1007FE00E4F0E8A3F0122D017464F50975080012F7
:10080E002BA6740C9007A5F8E4F0E8A3F0122D01C6
:10081E007464F509750800122BA6740D9007A5F8DF
:10082E00E4F0E8A3F0122D017464F50975080012C6
:10083E002BA6740E9007A5F8E4F0E8A3F0122D0194
:10084E007464F509750800122BA674029000AEF0C0
:10085E0090004FE0900072F090004FE0B4010874E9
:10086E000090007AF0801C90004FE0B402087400F3
:10087E009000BDF0800D90004FE0B4030674009020
:10088E0000CAF0D2170209769007A5E4F0A304F08F
:10089E00122D017464F509750800122BA6740290CE
:1008AE0007A5F8E4F0E8A3F0122D017464F50975BC
:1008BE000800122BA674039007A5F8E4F0E8A3F045
:1008CE00122D017464F509750800122BA67404909C
:1008DE0007A5F8E4F0E8A3F0122D017464F509758C
:1008EE000800122BA674059007A5F8E4F0E8A3F013
:1008FE00122D017464F509750800122BA67406906A
:10090E0007A5F8E4F0E8A3F0122D017464F509755B
:10091E000800122BA674079007A5F8E4F0E8A3F0E0
:10092E00122D017464F509750800122BA67401903E
:10093E0000AEF090004FE0900072F090004FE0B4E7
:10094E000108740090007AF0801C90004FE0B40211
:10095E000874009000BDF0800D90004FE0B40306C7
:10096E0074009000CAF0C217122FA69000B8E07063
:10097E0006740A9000B8F0900064E0700674E3907C
:10098E000064F0120198E5B54401F5B574069000C7
:10099E003EF0740190003FF07403900041F0740437
:1009AE00900042F0740E900043F07405900044F0F5
:1009BE00900040E0B404067404900044F074059076
:1009CE000045F0740090004AF0740090004BF074F3
:1009DE000190004CF0740090004DF074FF90004EAA
:1009EE00F0743390013CF0743690013DF0742D900C
:1009FE00013EF0743190013FF07420900140F0748C
:100A0E0034900141F07443900142F07479900143A7
:100A1E00F0746C900144F07420900145F0742090B5
:100A2E000146F07420900147F07420900148F07454
:100A3E0020900149F0742090014AF09000D4E0908B
:100A4E000061F090008BE0900062F090008CE090DE
:100A5E000063F0C212C21474C8900024F074C890DF
:100A6E000028F0C210C211A2B6B39209A2B3B3927B
:100A7E000A752600752500753746754C1E90005D6B
:100A8E00E4F075271975286490000874FFF0A374BC
:100A9E00DCF0C20D754B00C208752A007529009056
:100AAE00000CE4F0A3F0743A900765F074FD900723
:100ABE0066F0756D0090005EE4F0752C00752B00ED
:100ACE00900010E4F0A3F0900090E090000EF8E497
:100ADE00F0E8A3F0900071E075F032A4FFAEF09054
:100AEE00001EEEF0A3EFF090079FE0FEA3E0FF7470
:100AFE0003124C367401124C2890079DEEF0A3EFB2
:100B0E00F0754A0190003AE4F0C21FC21C756C00E9
:100B1E00753C00C20EC20FC220C203754D00C20446
:100B2E00D205C206D207C218C219D21A74FE90009C
:100B3E0035F074FE900036F0C21DD21E7538007569
:100B4E004400753A00753E32753F00754000743CA6
:100B5E00900038F0754100743C900039F0754200F9
:100B6E00754300900016E4F0A3F0754500D2B2D2A2
:100B7E00A4D2B0D2B1D2A3D2A7D2A6D2A5D2B790C8
:100B8E000071E0D394FA400674FA900071F07E0181
:100B9E007F00900063E0124C36900062E02FFF5011
:100BAE00010E900020EEF0A3EFF0EFD394FFEE9441
:100BBE000F4007900020E4F0A3F0900061E0700673
:100BCE0074FF900061F09000AEE0D3940240067482
:100BDE00019000AEF09000AFE07005754902800301
:100BEE007549039000B0E0D3940140067400900064
:100BFE00B0F09000B6E0C3940A5006740A9000B6A6
:100C0E00F09000C0E0700674019000C0F09000C03B
:100C1E00E0B4FF0674FE9000C0F09000C7E0D394DD
:100C2E00FE400674FE9000C7F074019000CDF07483
:100C3E00019000CEF074009000D0F074009000D5BA
:100C4E00F0D29CD2EC75CF01A298B3500302105C87
:100C5E00C298E54764046006E59964FF6002802A45
:100C6E00A21D4004D21D8020E547600874E625478A
:100C7E0090003AF0754700E546600874F0254690FE
:100C8E00003AF0754600C21D8002C21DE5476003A2
:100C9E00020D3C754700E599B4FF03754601E599D1
:100CAE00B4FE03754602E599B4FD03754603E59956
:100CBE00B4FC03754604E599B4FA03754605E59947
:100CCE00B4FB03754701E599B4F903754704E5993B
:100CDE00D394E54007E599C394F0400280168599B8
:100CEE00487547027E017F00E548C394E6124C36F4
:100CFE008E2F8F30753200753100E599D394C74031
:100D0E0007E599C394E64002801F8599487547030D
:100D1E0074E5C39548F530752F00AE2FAF3090496E
:100D2E00AC124BF77831124C71D29902105CE54738
:100D3E00B401028003020E14AE31AF329000651280
:100D4E004C5DE599F07831124C93AE31AF32EFB481
:100D5E000106EEB407028003020E14900765E0B49C
:100D6E003C028003020DFEC29C12041B12019890DD
:100D7E000061E09000D4F0900062E090008BF09063
:100D8E000063E090008CF0A2174032755001E550E0
:100D9E00D394075026E5509007A5F8E4F0E8A3F0A9
:100DAE0074AA900032F0122BD27464F50975080003
:100DBE00122BA67850740126F650D3803075500849
:100DCE00E550D3940E5026E5509007A5F8E4F0E8D0
:100DDE00A3F074AA900032F0122BD27464F5097548
:100DEE000800122BA67850740126F650D3122FA6A7
:100DFE0074C89007A5F8E4F0E8A3F0D29C754700FC
:100E0E007546007599FBE547B402028003020EB9E0
:100E1E00E5324531700685992E752D00AE31AF3213
:100E2E0074016F4E701BAC2DAD2EAA2FAB30ED2B77
:100E3E00FBEC3AFA8A068B07900065124C5DE59939
:100E4E00F07831124C93AE31AF3274026F4E705B4C
:100E5E00AC2DAD2E740D6D4C702C74639007A5F8EF
:100E6E00E4F0E8A3F074AB900032F0900072E090E2
:100E7E00004FF0122F0B900032E4F074C89007A5CB
:100E8E00F8E4F0E8A3F0AE2DAF2E74566F4E600C62
:100E9E0074486F4E600674666F4E700312041B1218
:100EAE000198854899754700754600E547B4033F9C
:100EBE00AE31AF32900065124C5DE599F07831128B
:100ECE004C93AE31AF32AC2FAD308F028E038C0609
:100EDE008D079049E8124BF7E493F9740193FEEAFB
:100EEE00D39EEB994009854899754700754600E5F4
:100EFE0047B40402800302105CAE31AF329000653D
:100F0E00124C5DE599F07831124C93AE31AF32EF61
:100F1E00B40006EEB40102800302105C12041B90B2
:100F2E000048E075F002A4FFAEF08F50EF90006520
:100F3E00124C68EFFCE0FDEC900068124C68EDFC82
:100F4E00E0FDEC2DFC900048E0B504028003021099
:100F5E004D0FEF900065124C68E550FFE0FCEF90EE
:100F6E000069124C68ECFFE0FCEFC39CFF90004858
:100F7E00E0B50702800302104DE550900067124C59
:100F8E0068E550FFE0FCEF90006A124C68ECFFE061
:100F9E00FCEF2CFF900048E0B50702800302104DD5
:100FAE00E55090006B124C68FFE0FCEF900048E0BB
:100FBE00F4042C90004FF0E55090006C124C68FF3A
:100FCE00E0FCEF900048E0F4042C900050F0E55067
:100FDE0090006D124C68FFE0FCEF900048E0F404C6
:100FEE002C900051F0E55090006E124C68FFE0FC22
:100FFE00EF900048E0F4042C9007A5F8E4F0E8A385
:10100E00F074AB900032F0122F0B7464F509750872
:10101E0000122BA69007A5124C44122F0B7464F5E8
:10102E0009750800122BA69007A5124C44122F0B1F
:10103E007599F97464F509750800122BA680FE7572
:10104E0099FF7464F509750800122BA680FEE5461B
:10105E006006A299B3B340030211DCC299E546B40F
:10106E00011FAE31AF3290003E124C5DE0F5997823
:10107E0031124C93AE31AF3274116F4E7003754610
:10108E0000E546B40203854A99E546B4031DAE3128
:10109E00AF32900065124C5DE0F599EFB40107EEAA
:1010AE00B407037546007831124C93E546B404023A
:1010BE00800302119EE53245317003852699AE31CB
:1010CE00AF3274016F4E7003853899AE31AF327402
:1010DE00026F4E7003853A99AE31AF3274036F4E84
:1010EE007003853E99AE31AF3274046F4E70038536
:1010FE004099AE31AF3274056F4E7003854199AE93
:10110E0031AF3274066F4E7003854299AE31AF32F5
:10111E0074076F4E7003854399AE31AF3274086F0A
:10112E004E7006900017E0F599AE31AF3274096F2C
:10113E004E7017A21EB340077599FAC21E800B900F
:10114E00003AE0F59990003AE4F0AE31AF32740A0D
:10115E006F4E7003854499AE31AF32740B6F4E7083
:10116E0003853F99AE31AF32740C6F4E70038545D7
:10117E0099AE31AF32740D6F4E70037599FC7831A4
:10118E00124C93AE31AF32740E6F4E700375460033
:10119E00E546B40539900040E0D394044010AE31DA
:1011AE00AF32904760124C5DE493F599800EAE31EC
:1011BE00AF32904844124C5DE493F599AE31AF32A4
:1011CE0074E36F4E70037546007831124C93E54709
:1011DE0064016005E547B40403020C53C28E7E1011
:1011EE007F00E53D124C36E58D75F010A4FDACF098
:1011FE00EF2DFDEE3CFCE58B75F01084FF7E00EDCF
:10120E002FFFEC3EFE8E278F28D28E900092E0604C
:10121E0056900018124C44900018E0FCA3E0FD908C
:10122E00001AE0FAA3E0FBEDB5033CECB50238B2D0
:10123E0016A208B34013A216B34008E5B54404F550
:10124E00B58006E5B554FBF5B590001AE0FEA3E0B7
:10125E00FF90001CE0FCA3E0FDEF2DFDEE3CFC90AA
:10126E00001AECF0A3EDF090009FE0600990009F53
:10127E00E0C394034002806F1244A6A208B3500943
:10128E0090005DE0C3944640028006900089E0F530
:10129E006BE56B75F005A4FFAEF09007A7EEF0A31B
:1012AE00EFF0900076E0C3953A4007E538C39539E4
:1012BE0050079007A7E4F0A3F0AE58AF599007A7D8
:1012CE00E0FCA3E0FDEFD39DEE9C4004C2A1800B99
:1012DE0090005DE0C394645002D2A190009FE0B4F0
:1012EE000205A2A1B392A290009FE0B4031C124586
:1012FE00C1AE58AF599007A7E0FCA3E0FDEFD39D18
:10130E00EE9C4004D2A18002C2A190007AE0600956
:10131E00A2B3300A01B3B340028039A2B3300A013E
:10132E00B34031A2B3300C01B3401C9000ADE0B419
:10133E000306A218B3B340028006740590003AF07B
:10134E00D218A20CB3920AA20CB330B301B340046C
:10135E00A20C920AA2B6300901B350030218DEA203
:10136E00B6300901B350030218DEA2B6300B01B33A
:10137E0050030217F5754A00900092E07013A20B0D
:10138E00B34008E5B554FBF5B58006E5B54404F564
:10139E00B50537A20DB3B35013AE27AF2890000892
:1013AE00E0FCA3E0FDEDC39FEC9E40030214B6E506
:1013BE0049B40330E537B42405754901801FA21FD7
:1013CE00B3401AE537C39424500690003A7401F0E6
:1013DE00E537D394244006740290003AF075370135
:1013EE00D21F805AE549B40206754901753724E5C6
:1013FE0037B42405753701804590003AE07030E52A
:10140E0037C39424500690003A7401F0E537D39414
:10141E00244006740290003AF0E537C3942450023B
:10142E00D21CE537D394244002D21CC296C29590AA
:10143E0000AFE0B4020512041B8003753701AE291C
:10144E00AF2AAC27AD28EF2DFDEE3CFC7403FF1246
:10145E004C188C298D2A900092E06043900018E081
:10146E00FEA3E0FF900092E08E048F05FF124C1851
:10147E0074018C068D07124C2890001CEEF0A3EF21
:10148E00F090001CE0F8A3E090001AC8F0A3C8F09A
:10149E00900018E4F0A3F0C216E5B554FBF5B5A222
:1014AE001CB34002C21C802BAE29AF2AAC27AD283C
:1014BE00EF2DFDEE3CFC74018C068D07124C288E30
:1014CE00298F2AAC27AD28EDD39488EC94134003D2
:1014DE0012041BE537B42412740390003AF0D21CA8
:1014EE009000AFE0B4020312041BAE2BAF2CAC275E
:1014FE00AD28EF2DFDEE3CFC8C2B8D2CAE27AF28AE
:10150E00EFD39DEE9C4011900010E0FAA3E0FBEBB0
:10151E00C394E8EA940340028006900010124C44F3
:10152E0090000CE0FEA3E0FFAC27AD28EF2DFDEE02
:10153E003CFC90000CECF0A3EDF09000AFE0B40298
:10154E001DAE27AF287405124C3674038E048F051A
:10155E00FF124C18900008ECF0A3EDF08016AE27A9
:10156E00AF287403124C367401124C28900008EE0A
:10157E00F0A3EFF0C28E758D00758B00753D007572
:10158E002801752700D28EE537240875F00984AF3F
:10159E00F07E00EF4E707590000CE0F8A3E0900026
:1015AE000AC8F0A3C8F090000AE0FEA3E0FFEF4ED9
:1015BE00600B7C7B7D89124B168E258F2690000C3E
:1015CE00E4F0A3F0AE25AF267428BE00039F5010A2
:1015DE00E53C2FFF50010E7401124C288E258F26EC
:1015EE0085263C9000B6E0A825B8000DD395264080
:1015FE0008E526900037F080099000B6E0149000C0
:10160E0037F0E54960067526007525009000ADE0BF
:10161E00B4030890002EE0653760028026A218B34E
:10162E004004D2198002B21990007AE0600BA21821
:10163E00B35006A219B3B340028006740490003A68
:10164E00F0C218E537640B6005E537B41D0990004C
:10165E009FE060031241E8900033E0653760079029
:10166E000034E0B53703754B00A20EB35006A20D41
:10167E00B3B3400302175D90006BE0B4015AE5402E
:10168E0075F00584FF7E00900565124C5DE0F53423
:10169E00753300AE33AF34900069E0124C3674648B
:1016AE008E048F05FF124C1874C18C068D07124CD8
:1016BE00368E358F3690000EE0FEA3E0FFAC33ADD4
:1016CE003412000374648E048F05FF124C189000C0
:1016DE000EECF0A3EDF0800F900069E075F0C1A460
:1016EE00FFAEF08E358F36E53AC394CC500690009F
:1016FE0069E07002805785F95085FA517E017F00AE
:10170E00E551124C36E5502FFF50010E8E338F34BB
:10171E00AC35AD36EF2DFDEE3CFC8C358D36D293CF
:10172E00D294E536F5FBE535F5FCE536F5E9E5351C
:10173E00F5EA9000ADE0B40314D291D292E536F5FD
:10174E00EBE535F5ECE536F5EDE535F5EED20EE5E6
:10175E0049B40106E537640B6002800F754C0190A9
:10176E00003D7401F0E5B54401F5B5E5497073909F
:10177E0000B2E0600D9000B9E0A825B800069526ED
:10178E00400280329000B2E0B4021790002CE06567
:10179E0037600790002DE0B53703754C0375450093
:1017AE00800CC200754500900016E4F0A3F0740999
:1017BE0090003AF0802C90002CE065376007900086
:1017CE002DE0B53703754C0190002CE0B53706902F
:1017DE00003D7401F090002DE0B5370674029000C4
:1017EE003DF0A20BB39209A20BB330B601B3500376
:1017FE000218DE754A01900092E07013A20BB340FE
:10180E0008E5B54404F5B58006E5B554FBF5B5A27B
:10181E000B9209E537D3944A4014D20DE537D39491
:10182E006E400B740390003AF0D21C753746900050
:10183E00BAE0B40107E543C39414400280031204D6
:10184E001B744690005DF0A204300501B35017A240
:10185E0004B34008E5B54408F5B58006E5B554F780
:10186E00F5B5A2049205A206300701B35017A206E1
:10187E00B34008E5B54402F5B58006E5B554FDF56F
:10188E00B5A2069207E543C394415009740E900029
:10189E003AF012041B900044E0FE900040E004C3B6
:1018AE009E4009900040E0D39406400974FB9000DE
:1018BE003AF012041B900049E06015900049E0FEDA
:1018CE00900043E06E600974FE90003AF012041B23
:1018DE00A21CB34004C296C295A210B3B350089096
:1018EE00002EE0653760030219C6A202B35006A2AD
:1018FE0000B3B340030219C29000ADE0B4030280FE
:10190E0003021997A208B34067A219B3402D120023
:10191E009EE536F5FBE535F5FCD293A203B3400206
:10192E00D2879000CBE0B402101200CBE536F5FB67
:10193E00E535F5FC75A700D287803312009EE5369B
:10194E00F5EBE535F5ECD291A203B34006E5B544CF
:10195E0010F5B59000CBE0B402141200CBE536F5CD
:10196E00EBE535F5EC75A700E5B54410F5B5801738
:10197E0012009EE536F5FBE535F5FCE536F5EBE5B3
:10198E0035F5ECD293D291802B12009EE536F5FB05
:10199E00E535F5FCD293A203B34002D2879000CB7B
:1019AE00E0B402101200CBE536F5FBE535F5FC751B
:1019BE00A700D287C210D211A211B3B35008900063
:1019CE002FE065376003021AA5A202B35006A200EB
:1019DE00B3B34003021AA19000ADE0B4030280033A
:1019EE00021A76A208B34067A219B3402D12009EC8
:1019FE00E536F5E9E535F5EAD294A203B34002D215
:101A0E00909000CBE0B402101200CBE536F5E9E57C
:101A1E0035F5EA75A700D290803312009EE536F5B3
:101A2E00EDE535F5EED292A203B34006E5B54420BE
:101A3E00F5B59000CBE0B402141200CBE536F5ED0F
:101A4E00E535F5EE75A700E5B54420F5B58017121E
:101A5E00009EE536F5E9E535F5EAE536F5EDE535D1
:101A6E00F5EED294D292802B12009EE536F5E9E582
:101A7E0035F5EAD294A203B34002D2909000CBE0A7
:101A8E00B402101200CBE536F5E9E535F5EA75A797
:101A9E0000D290D210C211E54CB40816123B17A218
:101AAE0010B35005A211B340028004D210D21175AA
:101ABE004C1EE54CB407061238CF754C08E54CB4F5
:101ACE00063D90000EE0FEA3E0FFEF4E6006A2087A
:101ADE00B3B340028023AE52AF5390000EE0FCA38E
:101AEE00E0FDEF2DFDEE3CFC8C528D53E537D3948B
:101AFE0012500690000E1200391236A1754C07E5F1
:101B0E004CB40506123501754C06E54CB404329002
:101B1E0000A0E0902B88F8282873123195801212BD
:101B2E003195800D12334380081233F58003123342
:011B3E00F5B1
:0F2B8800021B28021B2D021B32021B37021B3CB3
:101B3F00900082E060051242D18002C204754C050C
:101B4F00E54CB403028003021C39900085E0600568
:101B5F001243C18002C2069000A0E0D39402403F1E
:101B6F00900074E02403A825B8000495265009902E
:101B7F000076E0D3953A50028008D20274089000A4
:101B8F003AF0900074E0A825B80005D39526500BC5
:101B9F00900076E02403C3953A5002C20280399038
:101BAF000074E02403A825B8000495265007E538F3
:101BBF00C3953940028008D202740890003AF09021
:101BCF000074E0A825B80005D395265009E53924FF
:101BDF000FC395385002C2029000BAE07007E54378
:101BEF00C3941440028002D202A2024005754C0435
:101BFF00800A754C1E900016E4F0A3F0A208B340C3
:101C0F0029E54075F00584FF7E00900565124C5D57
:101C1F00E0C39469500512421D800F90079FE0F8B2
:101C2F00A3E090079DC8F0A3C8F0E54CB40A02806A
:101C3F0003021CD7900026E0C394465008C2967446
:101C4F0046900026F0900030E0B4011DE55A240ABA
:101C5F00F55A9007A1E0FEA3E0FF740A2FFF500191
:101C6F000E9007A1EEF0A3EFF0855A347533009074
:101C7F00002CE0F550120116E536900026F090008A
:101C8F0004E533F0A3E534F0E550900027F0C213DC
:101C9F009007A1E0F533A3E0F53490002CE0F55068
:101CAF00120116E536900024F0900000E533F0A302
:101CBF00E534F0E550900025F0C212E549B4010576
:101CCF00754C0B8003754C03900024E0B53773A25D
:101CDF0012404F900000E0FEA3E0FFEF4E6021AEF8
:101CEF0029AF2A900000E0FCA3E0FD120003740A64
:101CFF008E048F05FF124C18900000ECF0A3EDF04E
:101D0F00900025E0601A900000E0FEA3E0FFAC29F0
:101D1F00AD2AEF2DFDEE3CFC900000ECF0A3EDF0B2
:101D2F00D212AE27AF28900000E0FCA3E0FDEFC376
:101D3F009DEE9C400D1204DBD296C21274C8900027
:101D4F0024F0A212B3B35007900024E0B5370280FD
:101D5F000D1204DBD29674C8900024F0C2129000CA
:101D6F0026E0B53770A213404F900004E0FEA3E0C9
:101D7F00FFEF4E6021AE29AF2A900004E0FCA3E0F4
:101D8F00FD120003740A8E048F05FF124C18900089
:101D9F0004ECF0A3EDF0900027E0601A900004E04F
:101DAF00FEA3E0FFAC29AD2AEF2DFDEE3CFC900029
:101DBF0004ECF0A3EDF0D213AE27AF28900004E0AF
:101DCF00FCA3E0FDEFC39DEE9C400AC296744690C3
:101DDF000026F0C213A213B3B35007900026E0B54C
:101DEF003702800AC2967446900026F0C213E54C63
:101DFF00B40B028003021EB090002AE0C394465039
:101E0F00139000BBE0B40104C2968002C2957446E1
:101E1F0090002AF0900031E0B4011DE55A240AF534
:101E2F005A9007A1E0FEA3E0FF740A2FFF50010EA6
:101E3F009007A1EEF0A3EFF0855A347533009000B0
:101E4F002DE0F550120116E53690002AF0900006AD
:101E5F00E533F0A3E534F0E55090002BF0C2159078
:101E6F0007A1E0F533A3E0F53490002DE0F5501213
:101E7F000116E536900028F0900002E533F0A3E557
:101E8F0034F0E550900029F0C214E549B4010F7504
:101E9F00490074C8900024F074C8900028F0754C65
:101EAF0003900028E0B5377EA214404F900002E067
:101EBF00FEA3E0FFEF4E6021AE29AF2A900002E0B3
:101ECF00FCA3E0FD120003740A8E048F05FF124C71
:101EDF0018900002ECF0A3EDF0900029E0601A904A
:101EEF000002E0FEA3E0FFAC29AD2AEF2DFDEE3C92
:101EFF00FC900002ECF0A3EDF0D214AE27AF2890C7
:101F0F000002E0FCA3E0FDEFC39DEE9C401812041D
:101F1F00DB9000BBE0B40104D2968002D295C214CC
:101F2F0074C8900028F0A214B3B35007900028E0B3
:101F3F00B5370280181204DB9000BBE0B40104D265
:101F4F00968002D29574C8900028F0C21490002A8F
:101F5F00E0B5377BA215404F900006E0FEA3E0FFEF
:101F6F00EF4E6021AE29AF2A900006E0FCA3E0FD02
:101F7F00120003740A8E048F05FF124C189000068E
:101F8F00ECF0A3EDF090002BE0601A900006E0FE5D
:101F9F00A3E0FFAC29AD2AEF2DFDEE3CFC9000062F
:101FAF00ECF0A3EDF0D215AE27AF28900006E0FCC1
:101FBF00A3E0FDEFC39DEE9C40159000BBE0B40184
:101FCF0004C2968002C295744690002AF0C215A2F0
:101FDF0015B3B3500790002AE0B537028015900073
:101FEF00BBE0B40104C2968002C295744690002AE9
:101FFF00F0C215E54CB4020280030220A8123F8004
:10200F0012409790079DE0FEA3E0FF740A124C3632
:10201F0090000AE0FCA3E0FD74098F02FF124C1838
:10202F008D078C038E048A058B06124B169007A121
:10203F00EEF0A3EFF09000BBE0B401087478BE009F
:10204F00059F4002800D74789007A1F8E4F0E8A393
:10205F00F0801B9007A1E0FEA3E0FF74F0BE000329
:10206F009F500B74F09007A1F8E4F0E8A3F09007ED
:10207F00A1E0FEA3E0FFE55A2FFF50010E9007A14C
:10208F00EEF0A3EFF090003DE0B40103754C0A9021
:10209F00003DE0B40203754C0BE54CB401259000F4
:1020AF00D2E0902B97F8282873123D1E8012123D14
:1020BF001E800D123DA88008123E548003123E541C
:0F2B97000220B80220BD0220C20220C70220CCBB
:1020CF00754C029000BDE0B4020280030221EA9039
:1020DF000060E0D3953F5064900060E0F404253F2A
:1020EF00FE9000C0E08E00F5F0E884FF7E008F5078
:1020FF00EFC39410500CEF8550F0A4FDACF08D5051
:10210F0080037550FF900060E0D39550400B900016
:10211F0060E0C39550F54D8003754D009000DBE0F6
:10212F00D3954D40069000DBE0F54D9000DCE0C309
:10213F00954D50069000DCE0F54D8071900060E009
:10214F00C3953FFE9000C0E08E00F5F0E884FF7E5F
:10215F00008F50EFC39410500CEF8550F0A4FDACDE
:10216F00F08D5080037550FF85503475330090000B
:10217F0060E02534FFAE3350010E8E338F3474FF81
:10218F00BE0009D39F400585344D8003754DFF90E8
:10219F0000DBE0D3954D40069000DBE0F54D90005D
:1021AF00DCE0C3954D50069000DCE0F54DA208B37E
:1021BF00B350099000C8E0D3954E5002800A7407BF
:1021CF0090003AF0C297801375A710E5CDC3954DD7
:1021DF004004C2978002D29775A700E54BC39409BC
:1021EF004003022925A2EDB35003022925C2EDE5D4
:1021FF004B600302239990006EE0700302238890D6
:10220F0000A4E0B4010280030222E8900033E0B59D
:10221F00370280030222E57E017F00E5BE124C36B5
:10222F00E5BD2FFF50010E8E338F3490006EE0B45A
:10223F0001187410124C36900064E08E048F05FF65
:10224F00124C18ED900035F0802CAE33AF34741073
:10225F00124C36900064E08E048F05FF124C1890DC
:10226F000035E02DFD50010C74018C068D07124CCA
:10227F0028EF900035F0E54460089000CAE0640252
:10228F00600280219000CCE0B4011A900035E07517
:10229F00F0E7A4FFAEF0E5448E048F05FF124C1853
:1022AF00ED900035F0900035E0FE900036E0D39EC3
:1022BF004004D21A8002B21A900035E0900036F036
:1022CF009000A0E064016006A21AB3B3400280063A
:1022DF00900035E0F538022386D21A7E017F00E5A3
:1022EF00BE124C36E5BD2FFF50010E8E338F34904A
:1022FF00006EE0B401187410124C36900064E08E3A
:10230F00048F05FF124C18ED900035F0802CAE3382
:10231F00AF347410124C36900064E08E048F05FFBA
:10232F00124C18900035E02DFD50010C74018C06F5
:10233F008D07124C28EF900035F0E54460089000AF
:10234F00CAE06402600280219000CCE0B4011A90D0
:10235F000035E075F0E7A4FFAEF0E5448E048F057D
:10236F00FF124C18ED900035F09000A0E064016072
:10237F0006900035E0F538800375380090006AE06C
:10238F007005754B01800375BB18E54BB4010280D6
:10239F000302253B90006AE0700302252A7E017F2D
:1023AF0000E5BE124C36E5BD2FFF50010E8E338F68
:1023BF00349000B0E0B4010F7E0F7FFFAC33AD342B
:1023CF00124C8B8E338F349000D5E0B40245AE3370
:1023DF00AF34900020E0FCA3E0FDEDD39FEC9E40D6
:1023EF000A900020E533F0A3E534F0AE33AF34901C
:1023FF000022E0FCA3E0FDEFD39DEE9C400A90008D
:10240F0022E533F0A3E534F0AE33AF347404124C4D
:10241F00288F3A9000D5E0704CAE33AF3490002047
:10242F00E0FCA3E0FDEFD39DEE9C4009124C8B8E98
:10243F00338F348006753400753300AE33AF347488
:10244F0010124C36900061E08E048F05FF124C186D
:10245F008C338D347400D39D74019C400585343AC0
:10246F008003753AFF9000A0E0B4010280030225BB
:10247F0028A208B3B3500E900074E0A825B8000549
:10248F00D39526500302251D900075E075F019A411
:10249F00FFAEF09000B8E08E048F05FF124C18903D
:1024AF0000B1E0853AF0A4FFAEF074648D028C03A6
:1024BF008E048F05FF124C18EA2DFDEB3CFC8C337C
:1024CF008D34E544600F9000CAE0B402089000CC50
:1024DF00E0640160028017AE33AF3474E7124C36FC
:1024EF00E5448E048F05FF124C188C338D34900009
:1024FF0035E0A833B8000AD39534400585343880C9
:10250F000BA21AB34006900035E0F538800BA21AE3
:10251F00B34006900035E0F5388003753A0090001F
:10252F006DE07005754B02800375BB19E54BB40266
:10253F000280030225F690006DE070030225E5E5A9
:10254F0037D3941240030225E390001EE0FEA3E070
:10255F00FFE53E124C8390001EEEF0A3EFF07E01DC
:10256F007F00E5BE124C36E5BD2FFF50010E8E33B6
:10257F008F349000DAE07013740A124C3674518E57
:10258F00048F05FF124C188D3E8019AE33AF347493
:10259F000A124C368F048E057E017F95CDCCCD125D
:1025AF004B168F3EE53ED394644003753E64900016
:1025BF001EE0FEA3E0FFE53E2FFF50010E90001E30
:1025CF00EEF0A3EFF0900071E0048E048F05FF1280
:1025DF004C188D3E8003753E329000BDE07005753E
:1025EF004B03800375BB13E54BB4035E9000BDE056
:1025FF0060477E017F00E5BE124C36E5BD2FFF50D0
:10260F00010E8E338F347404124C288F3F9000BF0D
:10261F00E0853FF0A4FDACF07464FF124C188D3FC1
:10262F009000BEE0853FF0A4FFAEF074FF8E048FE4
:10263F0005FF124C188D4E8003753F0090006BE024
:10264F007005754B04800375BB17E54BB40402800E
:10265F00030226F790006BE0B4017C7E017F00E55A
:10266F00BE124C36E5BD2FFF50010E7404124C28DC
:10267F008E338F34900038E06012900038E0149061
:10268F004A2493A833B80006953440028006900080
:10269F0038E014F0900038E0C3947750139000386E
:1026AF00E004904A2493A833B80005D39534500220
:1026BF008006900038E004F0900038E0FE90009122
:1026CF00E08E0088F0A4FFAEF074648E048F05FFD7
:1026DF00124C188D40800375400090006CE070051F
:1026EF00754B05800375BB16E54BB40502800302DD
:1026FF00278A90006CE0B4017C7E017F00E5BE125A
:10270F004C36E5BD2FFF50010E7404124C288E334A
:10271F008F34900039E06012900039E014904A9D98
:10272F0093A833B80006953440028006900039E034
:10273F0014F0900039E0C394775013900039E004FF
:10274F00904A9D93A833B80005D395345002800664
:10275F00900039E004F0900039E0FE900097E08E91
:10276F000088F0A4FFAEF074648E048F05FF124C46
:10277F00188D41800375410075BB1FE54BB40633BF
:10278F007E017F00E5BE124C36E5BD2FFF50010ED6
:10279F008E338F347409124C3674E68E048F05FF16
:1027AF00124C188D43900073E07005754B07800332
:1027BF0075BB15E54BB4070280030228CC9000735C
:1027CF00E070030228BB7E017F00E5BE124C36E5A8
:1027DF00BD2FFF50010E8E338F347404124C288F8F
:1027EF0042900073E0B401159000C7E08542F0A459
:1027FF00FFAEF07407124C28EF9007AAF090007309
:10280F00E0B402159000C7E08542F0A4FFAEF0746B
:10281F0007124C28EF9007A9F0900073E0B4030261
:10282F0080030228B99000B4E0701CE542C3940AFB
:10283F005002D201E542D394644002C2019000934A
:10284F00E090005FF08063900093E070349000C7D9
:10285F00E08542F0A4FFAEF074FF8E048F05FF12E7
:10286F004C18ED90005FF0AE25AF26741EBE00062B
:10287F00D39F4002D201E53AD394E54002C20180D2
:10288F0029E542C3940A500DAE25AF26741EBE0033
:10289F0004D39F50028002D201E53AD394E540025F
:1028AF00C201900093E090005FF0800375420090AA
:1028BF0000CAE07005754B08800375BB14E54BB477
:1028CF0008509000CAE060397E017F00E5BE124CCF
:1028DF0036E5BD2FFF50010E8E338F34EFD3942189
:1028EF00EE940E40057544FF8015AE33AF3474106F
:1028FF00124C3674E38E048F05FF124C188D4480F2
:10290F000375440090006EE0600575BB1A80037577
:10291F00BB18054BD2ECAE27AF287428C39F742386
:10292F009E400C90005EE0C3943C4003022B85C296
:10293F000D7537469000AFE070057549028003753D
:10294F004903C293C294C291C292C287C290E5B5A5
:10295F0054EFF5B5E5B554DFF5B5C296C295C2A0F3
:10296F00C297C2A2C2A1E5B554BFF5B5E5B5547F74
:10297F00F5B5A21BB34008E5B54404F5B58006E5EF
:10298F00B554FBF5B5A20FB3500EE53AD3943340CF
:10299F0007E53AC394CC4003022A2DE5B54401F56F
:1029AF00B5744690005DF0900069E075F064A4FF87
:1029BF00AEF08E358F367402BE000AD39F40067577
:1029CF00360275350085F95085FA517E017F00E595
:1029DF0051124C36E5502FFF50010E8E338F34AC11
:1029EF0035AD36EF2DFDEE3CFC8C358D36D293D2C6
:1029FF0094E536F5FBE535F5FCE536F5E9E535F516
:102A0F00EA9000ADE0B40314D291D292E536F5EB23
:102A1F00E535F5ECE536F5EDE535F5EED20FE53AB2
:102A2F00C3941A5002C20F90000874FFF0A374DC15
:102A3F00F0900090E090000EF8E4F0E8A3F0C212DE
:102A4F00C21474C8900024F074C8900028F0C2100B
:102A5F00C211752600752500753C00C208756C0003
:102A6F00900016E4F0A3F0754C1E90079FE0FEA3B4
:102A7F00E0FF7403124C367401124C2890079DEE40
:102A8F00F0A3EFF0900082E060051242D18002C205
:102A9F0004900085E060051243C18002C206A204C3
:102AAF00300501B35017A204B34008E5B54408F54B
:102ABF00B58006E5B554F7F5B5A2049205A2063028
:102ACF000701B35017A206B34008E5B54402F5B5A8
:102ADF008006E5B554FDF5B5A2069207C203752C25
:102AEF0000752B00900010E4F0A3F0900071E075DA
:102AFF00F032A4FFAEF090001EEEF0A3EFF09000C6
:102B0F000CE4F0A3F0C21F90005EE0C3943C5010A1
:102B1F00E54BB4090990005EE004F0754B00803B73
:102B2F00E54BB40903754B00752800752700758DAB
:102B3F0000758B00753D0090005DE0C394645008F4
:102B4F0090005DE004F08006746490005DF09000EA
:102B5F005DE0B46406E5B554FEF5B590005EE0D3D4
:102B6F0094014007E543C3944140028009740E90DD
:092B7F00003AF012041B020C5391
:1049AC000000010001400160018001A001C001E094
:1049BC0002000300039603B603D603F404000500BB
:1049CC0005180530054805600578059005A805C053
:1049DC00060006140628063C066E068C00FF013FF6
:1049EC00015F017F019F01BF01DF01FF02FF039502
:1049FC0003B503D503F303FF04FF0517052F054784
:104A0C00055F0577058F05A705BF05FF061306276C
:104A1C00063B066F068B06A9DAD8D7D5D4D2D0CFF1
:104A2C00CDCBC9C7C6C4C2C0BEBCBAB8B5B3B1AF92
:104A3C00ADABA8A6A4A2A09D9B99969492908D8BA9
:104A4C0089878482807E7C79777573716F6D6B69D1
:104A5C00676563615F5D5B5957565452504F4D4BC0
:104A6C004A4847454442413F3E3C3B3A393736354C
:104A7C00343231302F2E2D2C2B2A29282726252570
:104A8C002423222121201F1E1E1D1C1C1B1A1A1937
:104A9C0019EEECEBEAE9E8E7E5E4E3E1E0DEDDDB87
:104AAC00D9D8D6D4D2D0CECCCAC8C6C3C1BFBCBA52
:104ABC00B7B5B2B0ADABA8A5A3A09D9B98959290AD
:104ACC008D8A8785827F7D7A7775726F6D6A68654E
:104ADC0063615E5C5A575553514F4D4B49474543A3
:104AEC0042403E3C3B393836353332312F2E2D2B5C
:104AFC002A292827262524232221201F1E1D1D1C80
:0A4B0C001B1A1A19181817161615AF
:102BA600750B00750A00AE0AAF0BAC08AD09EDC394
:102BB6009FEC9E401674FF124C0875CF01780B747B
:102BC6000126F6500418E436F650DB22900032E077
:102BD600B4AA1C900765E0B43C159007A5E0FEA3D7
:102BE600E0FFEF4E6009741EBE0004D39F5003023F
:102BF6002D0075360075350075F8099007A5E0FEBD
:102C0600A3E0FF74076F4E6006740E6F4E70067475
:102C16003A900765F09007A5E0FEA3E0FF7408BEB2
:102C2600001ED39F401A7E017F089007A5E0FCA3F3
:102C3600E0FD1DBDFF011C1200038E338F34801F83
:102C46009007A5E0FEA3E0FF7408124C838F048E64
:102C5600057E017F08CDCCCD1200038E338F34AEB6
:102C660035AF36740CD39F74019E5003022CFBA221
:102C7600F9B3407EE5364535700375A382AE35AFB0
:102C86003674016F4E700375A300AE35AF3674020D
:102C96006F4E700D9007A6E075F002A4FDACF08DA6
:102CA600A3AE35AF3674036F4E700375A300AE3511
:102CB600AF367403BE00039F5013AC33AD34ED2F13
:102CC600FFEC3EFE900061124C5DE0F5A3AE35AF21
:102CD60036EFB40B09EEB401057414124C08AE3588
:102CE600AF36EFB40B07EEB4010375F80D78351265
:102CF6004C93022C65900032E4F02275360075354F
:102D06000075F8099007A5E0FEA3E0FF7408BE0071
:102D16001ED39F401A7E017F089007A5E0FCA3E022
:102D2600FD1DBDFF011C1200038E338F34801F90E2
:102D360007A5E0FEA3E0FF7408124C838F048E05FE
:102D46007E017F08CDCCCD1200038E338F34AE3595
:102D5600AF367411D39F74019E5003022E31A2F92F
:102D6600B35003022E2EE5364535700375A3D2AE59
:102D760035AF3674016F4E700375A300AE35AF36AE
:102D860074026F4E700D9007A6E075F002A4FDACBC
:102D9600F08DA3AE35AF3674036F4E700375A30086
:102DA600AE35AF3674046F4E700375A300AE35AF03
:102DB6003674056F4E700375A300AE35AF367406D4
:102DC6006F4E700375A300AE35AF3674076F4E7045
:102DD6000375A300AE35AF3674086F4E700375A346
:102DE60000AE35AF367408BE00039F5016AC33AD47
:102DF60034ED2FFFEC3EFE90005C124C5DE5A3F037
:102E060075A300AE35AF36EFB41009EEB401057404
:102E160014124C08AE35AF36EFB41007EEB401030A
:102E260075F80D7835124C93022D542275360075BF
:102E3600350075F809AE35AF367417BE0004D39F5A
:102E46005003022F0AA2F9B35003022F07E53645B5
:102E560035700375A3D2AE35AF3674016F4E70036D
:102E660075A300AE35AF3674026F4E700D9007A68F
:102E7600E075F002A4FDACF08DA3AE35AF36740359
:102E86006F4E700375A300AE35AF3674046F4E7087
:102E96000375A300AE35AF3674056F4E700375A388
:102EA60000AE35AF3674066F4E700375A300AE35AF
:102EB600AF3674076F4E700375A300AE35AF367428
:102EC600086F4E700375A300AE35AF367408BE00AA
:102ED600039F500C900046124C5DE5A3F075A300CD
:102EE600AE35AF3674166F4E70057414124C08AEBC
:102EF60035AF3674166F4E700375F80D7835124C73
:102F060093022E3B22900032E0B4AB028003022FE4
:102F1600A575360075350075F809AE35AF367412ED
:102F2600BE007CD39F4078A2F9B34070E5364535A4
:102F3600700375A382AE35AF3674016F4E7003759C
:102F4600A300AE35AF3674026F4E700D9007A6E043
:102F560075F002A4FDACF08DA3AE35AF3674036FE9
:102F66004E700375A300AE35AF367403BE00039FE3
:102F7600500990004B124C5DE0F5A3AE35AF3674A8
:102F8600116F4E70057414124C08AE35AF367411BD
:102F96006F4E700375F80D7835124C93022F202270
:102FA60090003BE4F074649007A5F8E4F0E8A3F021
:102FB600122E3274C89007A5F8E4F0E8A3F090004A
:102FC60052E0B4371A90004FE0900046F09000505F
:102FD600E0900047F0900051E0900048F080469065
:102FE600003B7401F074659007A5F8E4F0E8A3F0DF
:102FF600122E3274C89007A5F8E4F0E8A3F090000A
:1030060052E0B4371A90004FE0900046F09000501E
:10301600E0900047F0900051E0900048F080067480
:103026000290003BF090003CE4F074669007A5F82F
:10303600E4F0E8A3F0122E3274C89007A5F8E4F085
:10304600E8A3F0900051E0B4371290004FE09000F2
:1030560040F0900050E0900049F0807690003C747B
:1030660001F074679007A5F8E4F0E8A3F0122E3299
:1030760074C89007A5F8E4F0E8A3F0900051E0B416
:10308600371290004FE0900040F0900050E0900022
:1030960049F0803E740290003CF074689007A5F8F1
:1030A600E4F0E8A3F0122E3274C89007A5F8E4F015
:1030B600E8A3F0900051E0B4371290004FE0900082
:1030C60040F0900050E0900049F0800674039000B4
:1030D6003CF022E55D2534FFAE3350010E900065CD
:1030E600124C5DE0F55EE55D2534FFAE3350010E12
:1030F6000FBF00010E900065124C5DE0F55F85651F
:1031060061E55EB55F05855E5D8041E55FD3955EF1
:10311600401DE55FC3955E8560F0A4FFAEF0E561F6
:103126008E048F05FF124C18ED255EF55D801DE5BA
:103136005EC3955F8560F0A4FFAEF0E5618E048FF7
:1031460005FF124C18EDF404255EF55D22E55FD30C
:10315600955E401DE55FC3955E8560F0A4FFAEF009
:10316600E5618E048F05FF124C18ED255EF55D8036
:103176001DE55EC3955F8560F0A4FFAEF0E5618E48
:10318600048F05FF124C18EDF404255EF55D22E56B
:103196003875F00484FF7E008F5DE53875F0048491
:1031A600ADF07C008D60756504753301753400E5FE
:1031B6005DC3943F50051230D980069001A4E0F516
:1031C6005D855D53755200900037E075F020A4FFD1
:1031D600AEF09000B6E08E048F05FF124C188D5DA0
:1031E60090009EE0D39538500302329B9000C2E0D7
:1031F600D395384010ED9001A5124C68E0F5557551
:10320600540002329890008DE0D395384043E55D36
:103216009001A5124C68E0F55EE55D9001C5124C83
:1032260068E0F55F9000C2E0F4042538F560900090
:103236008DE0FE9000C2E0F4042EF561E55EB55F18
:1032460005855E5D8003123153855D55755400809A
:1032560041E55D9001C5124C68E0F55EE55D9001C3
:10326600E5124C68E0F55F90008DE0F4042538F532
:103276006090009EE0FE90008DE0F4042EF561E57E
:103286005EB55F05855E5D8003123153855D5575BC
:1032960054000233429000C5E0D395385011E55DE5
:1032A600900225124C68E0F55575540002334290A1
:1032B600008EE0D395385043E55D900205124C68C8
:1032C600E0F55EE55D900225124C68E0F55F900042
:1032D6008EE0F4042538F5609000C5E0FE90008E7F
:1032E600E0F4042EF561E55EB55F05855E5D80035D
:1032F600123153855D557554008041E55D9001E5B9
:10330600124C68E0F55EE55D900205124C68E0F54A
:103316005F90009EE0F4042538F56090008EE0FE94
:1033260090009EE0F4042EF561E55EB55F05855ECE
:103336005D8003123153855D55755400229000D689
:10334600E0F562756511753302753400AE25AF265A
:10335600E56275F00FA4FDACF0EDD39FEC9E402125
:10336600E5628E048F05FF124C18ED75F010A4FF70
:10337600AEF0E53875F01184FD7C00ED2FF5638025
:103386000EE53875F01184FF7E00EF24F0F56385B5
:10339600635DE53875F01184AFF07E008F60123002
:1033A600D9855D64AE25AF269000D6E075F00FA4F2
:1033B600FDACF0EDD39FEC9E4028753302753410BA
:1033C60085635D1230D985645E855D5FAE25AF2667
:1033D600E5628E048F05FF124C518D608562611285
:1033E6003153855D537552007555647554002290AE
:1033F60000D6E0F562756511753302753400AE25A9
:10340600AF26E56275F00FA4FDACF0EDD39FEC9E00
:103416004021E5628E048F05FF124C18ED75F01001
:10342600A4FFAEF0E53A75F01184FD7C00ED2FF5B2
:1034360063800EE53A75F01184FF7E00EF24F0F507
:103446006385635DE53A75F01184AFF07E008F60A9
:103456001230D9855D64AE25AF269000D6E075F0B2
:103466000FA4FDACF0EDD39FEC9E4028753302759A
:10347600341085635D1230D985645E855D5FAE2547
:10348600AF26E5628E048F05FF124C518D60856272
:1034960061123153855D537552009000A0E0B4046B
:1034A60053E53875F00484FF7E008F5DE53875F0CE
:1034B6000484ADF07C008D60756504753301753448
:1034C60000E55DC3943F50051230D980069001A4F3
:1034D600E0F55DAE52AF53E55D124C3674648E0472
:1034E6008F05FF124C18AE52AF53EF2DFDEE3CFC8C
:1034F6008C528D537555647554002290006BE0B460
:103506000146E54075F00584FF7E008F5DE5407558
:10351600F00584ADF07C008D607565057533057525
:103526003400E55DC3941750051230D98006900526
:103536007CE0F55DAE54AF55E55D2FFF50010E748E
:1035460064124C838E548F5590006CE0B40146E5AE
:103556004175F00584FF7E008F5DE54175F00584B9
:10356600ADF07C008D60756505753305753448E5ED
:103576005DC3941750051230D980069005C4E0F556
:103586005DAE54AF55E55D2FFF50010E7464124CCD
:10359600838E548F5590007BE0B40249E543C39473
:1035A6004175F00584FF7E008F5DE54375F0058467
:1035B600ADF07C008D60756505753306753400E5E4
:1035C6005DC3941350051230D98006900678E0F555
:1035D6005DAE54AF55E55D2FFF50010E7464124C7D
:1035E600838E548F559000BDE0B4020280030236EC
:1035F600A0E53875F01584FF7E008F5DE53875F01F
:103606001584ADF07C008D607565157533037534D2
:10361600F4E55DC3940B50051230D980069004641E
:10362600E0F55DE55D75F0FFA4FFAEF09000BEE04D
:103636008E048F05FF124C18ED900060F0E53F7583
:10364600F078A4FFAEF074FF8E048F05FF124C18BD
:103656008C338D3474028C068D07124C288F5DAC2A
:1036660033AD347404FF124C518D607565047533A7
:103676000675346EE55DC3941D50051230D980067B
:103686009006F0E0F55DAE54AF55E55D2FFF5001B5
:103696000E7464124C838E548F5522900073E0B4DE
:1036A60001179007AAE02555FFAE5450010E900071
:1036B600C7E0124C838E548F55900073E0B4031606
:1036C600A201B3B3501090005FE0C39405A825B8DB
:1036D6000006952640028010900095E02555FFAE25
:1036E6005450010E8E548F5590006DE0B402028046
:1036F600030238CE900070E0602FE540D3941E4060
:1037060028900010E0FEA3E0FF9000ABE075F00308
:10371600A4FDACF0EFD39DEE9C400E9000CFE0A848
:1037260025B80005D3952650030238CE9000B8E0A0
:103736008538F0A4FFAEF07405124C367407124CAF
:10374600288E338F34900077E0A825B8000495269C
:103756005012900078E075F002A4FDACF0EFC39D26
:10376600EE9C40030238CEE53875F00B84FF7E00F0
:103776009005F5124C5DFEE0FFEE90006FE0FEEF67
:103786008E0088F0A4FFAEF074648E048F05FF12DD
:103796004C188C338D34900037E075F018A4FFAECA
:1037A600F09000B6E08E048F05FF124C188C068D43
:1037B6000790060D124C5DAE33AF34E0124C3674F2
:1037C600648E048F05FF124C188C338D34E53EA8A9
:1037D60033B80077D395344072E53EC39534FFE4A1
:1037E6009533FE8E338F347428BE00039F500C75BC
:1037F6003428753300740D90003AF0AE33AF349030
:103806000070E0124C3674288E048F05FF124C1897
:103816008C338D34AE52AF53740A8E048F05FF126B
:103826004C188D068C07AC33AD34CFCECF120003C7
:10383600740A8E048F05FF124C188C338D34AE52E9
:10384600AF53124C8B8E528F53807DE53EA833B812
:10385600000495345072AE33AF34E53E124C838E7D
:10386600338F347428BE00039F500C75342875338B
:1038760000740D90003AF0AE33AF34900070E01251
:103886004C3674288E048F05FF124C188C338D34F9
:10389600AE52AF53740A8E048F05FF124C188D0674
:1038A6008C07AC33AD34CFCECF120003740A8E042E
:1038B6008F05FF124C188C338D34AE52AF53EF2D5B
:1038C600FDEE3CFC8C528D5322AE52AF53AC54AD40
:1038D6005512000374648E048F05FF124C188C5227
:1038E6008D53900068E08C068D07124C3674648EFA
:1038F600048F05FF124C188C528D53A2084017AE48
:1039060025AF267405BE00039F5002D208E53AD3C0
:1039160094CC4002D2029000CAE0B402089000CCD7
:10392600E0640160028017AE52AF53E544124C3694
:1039360074E78E048F05FF124C188C528D5390003D
:103946008AE05402601B900081E0A825B80012D3DB
:103956009526400DA208B3B35007E53AC3949A40A2
:10396600028028AE5BAF5C90007FE075F002A4FD9C
:10397600ACF0EF2DFDEE3CFC74022DFD50010CE584
:103986003ABC0007D39D4003756901853A5C755BB7
:1039960000E5697003023A259000DDE0C3956940B1
:1039A60070E54075F00584FF7E00900565124C5D5C
:1039B600E0F534753300AE33AF3490008FE0124C2F
:1039C6003674648E048F05FF124C188C358D369034
:1039D60000DDE004C395698C068D07124C36900015
:1039E600DDE08E048F05FF124C188C358D36900065
:1039F60080E08C068D07124C36740A8E048F05FF04
:103A0600124C18AE52AF53EF2DFDEE3CFC8C528D8E
:103A16005305699000DDE0C3956950037569009010
:103A2600008AE05401601B90007EE0A825B80012D1
:103A3600D39526400DA208B3B35007E538C394CCFE
:103A46004002802590007CE075F003A4FFAEF0E50F
:103A5600662FFF50010E74032FFF50010EE538BE8E
:103A66000007D39F4003756A01853866E56A7003CF
:103A7600023B009000DEE0C3956A4070E54075F0B9
:103A86000584FF7E00900565124C5DE0F5347533C4
:103A960000AE33AF3490008FE0124C3674648E045F
:103AA6008F05FF124C188C358D369000DEE004C36E
:103AB600956A8C068D07124C369000DEE08E048FD8
:103AC60005FF124C188C358D3690007DE08C068DE6
:103AD60007124C36740A8E048F05FF124C18AE522C
:103AE600AF53EF2DFDEE3CFC8C528D53056A9000D2
:103AF600DEE0C3956A5003756A0090008FE0A85215
:103B0600B800049553500990008FE0F553755200A4
:103B1600229000CBE0B401028003023C22A208B34B
:103B26005003023C20900096E0B40168AE52AF53B9
:103B3600AC25AD26120003743C8E048F05FF124C93
:103B4600189000A6E0BC00109D400D9000A8E0A8CB
:103B560052B8000495535002D203AE52AF53AC256F
:103B6600AD26120003743C8E048F05FF124C18908C
:103B760000A6E0C3940ABC0015D39D40119000A88E
:103B8600E0C39405A852B80005D3955350028002AD
:103B9600C2038068AE52AF53AC25AD261200037443
:103BA600788E048F05FF124C189000A6E0BC00101A
:103BB6009D400D9000A8E0A852B80004955350040B
:103BC600D2038038AE52AF53AC25AD261200037433
:103BD600788E048F05FF124C189000A6E0C3940A55
:103BE600BC0015D39D40119000A8E0C39405A852CF
:103BF600B80005D3955350028002C203A203B34016
:103C060019AE52AF539000A7E0124C3674648E047E
:103C16008F05FF124C188C528D538002C203900000
:103C2600CBE0B40258E53875F00884FF7E008F5D5E
:103C3600E53875F00884ADF07C008D607565087513
:103C460033017534E0E55DC3943F50051230D980E9
:103C560006900264E0F55DE55D75F05EA4FFAEF0EA
:103C6600740A8E048F05FF124C188C568D577402F9
:103C7600BC000AD39D4006755702755600A200B3D4
:103C86004006A202B3B35009900016E4F0A3F080F8
:103C960024AE52AF537400D39F74019E400C900023
:103CA60016E552F0A3E553F0800B74FF900016F86A
:103CB600E4F0E8A3F09000ADE0D394024006A20839
:103CC600B3B34002800DAE52AF537402124C368E1F
:103CD600528F53900096E0B4010DAE52AF5374026A
:103CE600124C368E528F53AE52AF53745E124C3610
:103CF600740A8E048F05FF124C188C528D53740271
:103D0600BC000AD39D4006755302755200900014FC
:103D1600E552F0A3E553F022900037E090036512D8
:103D26004C68E0F567756864900037E0FE9000A186
:103D3600E0D39E4037E53875F00884FF7E008F5D3E
:103D4600E53875F00884ADF07C008D607565087502
:103D56003303753496E55DC3941F50051230D98040
:103D66000690041AE0F55D855D688035E53875F0E6
:103D76000884FF7E008F5DE53875F00884ADF07C21
:103D8600008D607565087533037534B6E55DC394BB
:103D96001F50051230D9800690043AE0F55D855D26
:103DA60068229000D7E0F5627565117533047534A5
:103DB60000AE25AF26E56275F00FA4FDACF0EDD39D
:103DC6009FEC9E4021E5628E048F05FF124C18ED94
:103DD60075F010A4FFAEF0E53875F01184FD7C0097
:103DE600ED2FF563800EE53875F01184FF7E00EF48
:103DF60024F0F56385635DE53875F01184AFF07ED8
:103E0600008F601230D9855D64AE25AF269000D74D
:103E1600E075F00FA4FDACF0EDD39FEC9E40287545
:103E2600330475341085635D1230D985645E855D13
:103E36005FAE25AF26E5628E048F05FF124C518DCD
:103E460060856261123153855D67756864229000F2
:103E5600D7E0F562756511753304753400AE25AF8C
:103E660026E56275F00FA4FDACF0EDD39FEC9E4005
:103E760021E5628E048F05FF124C18ED75F010A433
:103E8600FFAEF0E53A75F01184FD7C00ED2FF56389
:103E9600800EE53A75F01184FF7E00EF24F0F5639D
:103EA60085635DE53A75F01184AFF07E008F601290
:103EB60030D9855D64AE25AF269000D7E075F00F4A
:103EC600A4FDACF0EDD39FEC9E4028753304753409
:103ED6001085635D1230D985645E855D5FAE25AF62
:103EE60026E5628E048F05FF124C518D6085626156
:103EF600123153855D677568649000D2E0B4047929
:103F0600900037E0FE9000A1E0D39E4037E538757B
:103F1600F00884FF7E008F5DE53875F00884ADF00B
:103F26007C008D60756508753303753496E55DC351
:103F3600941F50051230D9800690041AE0F55D856D
:103F46005D688035E53875F00884FF7E008F5DE595
:103F56003875F00884ADF07C008D607565087533A2
:103F6600037534B6E55DC3941F50051230D980063B
:103F760090043AE0F55D855D682290006BE0B4013F
:103F86003BE54075F00584FF7E008F5DE54075F0EA
:103F96000584ADF07C008D60756505753305753457
:103FA60018E55DC3941750051230D9800690059424
:103FB600E0F55DE568255DC39464F56890006CE006
:103FC600B4013BE54175F00584FF7E008F5DE54158
:103FD60075F00584ADF07C008D607565057533055B
:103FE600753460E55DC3941750051230D98006908C
:103FF60005DCE0F55DE568255DC39464F568E56775
:104006002568F55A900073E0B402109007A9E025E0
:104016005AFE9000C7E0F4042EF55A9000CAE0D389
:1040260094014040E544C394E7501D74E7C39544AA
:10403600FE9007ABE08E00F5F0E884FF7E008F5D12
:10404600E55A255DF55A801CE544C394E7FE9007C2
:10405600ABE08E00F5F0E884FF7E008F5DE55AC385
:10406600955DF55AA2084006E5672464F55AE55AB7
:10407600D394644009E55AC39464F55A8003755A8B
:10408600009000A3E0C3955A50069000A3E0F55AAD
:1040960022D2009000B9E0A825B800049526503B2E
:1040A6009000B9E0A825B8000495265003755A0F6C
:1040B6009000B9E004A825B8000495265003755A67
:1040C6000A9000B9E02402A825B8000495265005F8
:1040D600755A05C200740990003AF07E017F00907F
:1040E60000A9E0124C369000B8E08E048F05FF124E
:1040F6004C18E538BC000CD39D4008C200740A90E9
:10410600003AF09000AAE0C39540500D9000BCE044
:10411600A825B80006952640028008C200740B90B8
:10412600003AF0A2004003755A05900073E0B4030C
:1041360006A201B3B34002802B90005FE0C3940552
:10414600A825B800049526500C900094E0F55A7402
:104156000C90003AF090005FE0A825B80004952680
:104166005002C200855A45900065E0255AFE90002F
:1041760037E075F01E84FC7F00EE2CF55A22900085
:1041860037E075F00584FF7E008F5D900037E0759F
:10419600F00584ADF07C008D60756505753303759B
:1041A60034D69000B6E01475F00584FF7E00E55D18
:1041B600BE00039F50051230D9800BE55D90043B8D
:1041C600124C68E0F55DE55D9007ACF09007ACE059
:1041D600FE9000A5E0C39E50089000A5E09007ACB5
:1041E600F022E54075F00584FF7E00900565124CCF
:1041F6005DE0F56CE56CD394644010E56CC39464A3
:1042060075F00F84FF7E008F6C8003756C00900044
:1042160088E0256CF56C2290079FE0FEA3E0FF7412
:1042260004124C28E538124C36740F8E048F05FFA5
:10423600124C1890079DECF0A3EDF090007BE0B4D3
:104246000262E543C3944175F00584FF7E008F5DED
:10425600E54375F00584ADF07C008D6075650575E8
:104266003306753414E55DC3941750051230D980B2
:104276000690068CE0F55D90079DE0FEA3E0FF74D6
:104286000A8E048F05FF124C18E55D8C068D071209
:104296004C36740A8E048F05FF124C1890079DEC5D
:1042A600F0A3EDF090079DE0FEA3E0FF9007A3E0EA
:1042B600FCA3E0FDEDD39FEC9E400F9007A3E0F832
:1042C600A3E090079DC8F0A3C8F022900082E0B456
:1042D6000103852650900082E0B402129000B8E0F7
:1042E6008538F0A4FFAEF07408124C288F50900069
:1042F60082E0B40303853A50900082E0B40403855B
:104306004050900082E0B40507E541C39414F5508F
:10431600900082E0B40603854250900082E0B40724
:1043260003854350900082E0B40803854450900012
:1043360082E0B40903853F50900083E0FE9000843C
:10434600E0D39E404B900082E0B40418900084E0D5
:10435600C395505002D204900083E0D3955040029A
:10436600C204802A900083E0C395505009900084CF
:10437600E0D3955050028002D204900083E0D3959A
:10438600505009900084E0C395505002C204802A20
:10439600900083E0D395504009900084E0C3955087
:1043A60040028002C204900083E0C3955040099009
:1043B6000084E0D395504002D20422900085E0B4F8
:1043C6000103852650900085E0B402129000B8E003
:1043D6008538F0A4FFAEF07408124C288F50900078
:1043E60085E0B40303853A50900085E0B404038564
:1043F6004050900085E0B40507E541C39414F5509C
:10440600900085E0B40603854250900085E0B4072D
:1044160003854350900085E0B4080385445090001E
:1044260085E0B40903853F50900086E0FE90008742
:10443600E0D39E4040900086E0C39550500990001E
:1044460087E0D3955050028002D206900086E0D3D2
:1044560095505009900087E0C395505002C20690CF
:104466000085E0B401099000C4E0D3953A5002807B
:1044760002C206802A900086E0D39550400990003B
:1044860087E0C3955040028002C206900086E0C3D2
:1044960095504009900087E0D395504002D20622FD
:1044A600AE58AF5974F5D39F74019E4008785812E0
:1044B6004C930245C0755901755800AE25AF26E5E7
:1044C6006CBE000DD39F400990009AE0D3956D40D5
:1044D600028023756D00E56CC39526F55090009D0E
:1044E600E0D3956B4008E56B2550F56B8006900090
:1044F6009DE0F56B8002056D900076E0D3953A401D
:104506001CE538C395394015AE25AF26E56CBE00CF
:10451600039F500990009BE0D3956E4002806E90F9
:1045260007ADE0A825B800049526500375700090E5
:1045360007ADE0A825B8000BD395264006E52690E2
:1045460007ADF0E5707041E526C3956CF550E55072
:10455600D39405400375500590009CE0C3956B50BD
:1045660007E550C3956B40028009E56BC39550F58E
:104576006B800690009CE0F56B90009CE0D3956BF9
:10458600400690009CE0F56B756E008002056EE5B6
:10459600707016900076E0C3953A500DE56C2405D0
:1045A600A825B8000695264002800F900089E0F500
:1045B6006B75700174789007ADF022AE58AF5974E0
:1045C600E9D39F74039E40087858124C9302475FC4
:1045D600755901755800756B32A220402A756B1902
:1045E600900089E075F002A4FFAEF0E56DBE00060E
:1045F600D39F4002D220056D75700374789007AD85
:10460600F0756F0002474EAE25AF26E56C6F4E7013
:104616000302474EE56CBE000DD39F400990009AF9
:10462600E0D3956D4002800F756D00E570C394036D
:104636005003756B19800DE56CC39526F550E56D35
:104646002550F56D900076E0D3953A400E9007AD73
:10465600E0A825B80007D395264002800C056F9088
:104666000089E0B56F03757000E570B40306A20813
:10467600B3B34002800A056FE56FB43C0375700260
:10468600E570B402299007ADE0A825B8000ED395D1
:10469600264009E5269007ADF0756F00900076E09C
:1046A600C3953A5009756F0074789007ADF0E570C0
:1046B600705A900076E0D3953A401CE538D3953988
:1046C6004015AE25AF26E56CBE00039F500990004D
:1046D6009BE0D3956E40028008756E00756B4B802B
:1046E60028E526C3956CF550E550D394054003752F
:1046F6005005900076E0D3953A4008E56E2550F5D2
:104706006E8006E56E2406F56E756F00E570701610
:10471600900076E0C3953A500DE56C2405A825B8BF
:104726000006952640028003757001E570B40118F5
:10473600756B19056F900089E0B56F067570027587
:104746006F0074789007ADF0E56B75F00AA4FFAEC4
:0A475600F09007A7EEF0A3EFF022A9
:094C68002582F582500205832229
:0F008C0025E050020583258250020583F582226C
:104BF700EF2F500205832582F582E5833E2EF5834C
:014C0700228A
:104C8300CFC39FFF50011E22C3EF9DFFEE9CFE2268
:094C7100E493F608740193F622A5
:084C93000806B6000218062213
:0D4C4400A3E004F07006120049E004F02225
:0E003900A3E014F0B4FF06120049E014F02218
:0E4C2800048007C3CE13CECF13CFD5E0F62203
:104B1600BC000FBE0008ED8FF084FFADF022E4FE6E
:104B2600FF22BE000DEF60FE54F0606F20E7030227
:104B36004BCCEAC0E0EBC0E078017A0075F001EEFC
:104B460020E710EF25E0FFEE33FE0AC5F023C5F09F
:104B560030E7F0EA5407F9096A7A007B0060010839
:104B6600C3EC9E40167004ED9F4010ED9FFDEC9E39
:104B7600FCE5F0CA4ACA03F5F08005E5F003F5F056
:104B8600C3EE13FEEF13FFD9D77908CACBCAD8D024
:104B9600EAFEEBFFD0E0FBD0E0FA22EC8FF084FCDB
:104BA600ED54F045F0C48FF084FEEDC454F045F0AA
:104BB600C48FF084FDEEC4FE54F02DFFEE540F3C7E
:104BC600FEADF07C0022790078008FF0EC7E0820A4
:104BD600E70DC3CD33CD33C933C9C833C8DEF0843E
:104BE60049F9E5F08FF0BE00E6FD7C00E9FFE8FE3E
:014BF600229C
:0E4C3600F88FF0A4FFE5F0CE88F0A42EFE2249
:10000300EF8DF0A4F9A8F0EF8CF0A428F8EE8DF0B2
:06001300A428FEE9FF2213
:104C0800600D782B024C12007830D8FED5E0F822DF
:104C1800EEC0E07E00124B16EFFDEEFCD0E0FE2267
:0C4C5100EEC0E07E00124B16D0E0FE2208
:03001B0002001EC2
:0300530002005652
:03009B00020071EF
:03000000024C7A35
:094C7A0075817175D0000205BDC1
:0B4C5D00E5822FF582E5833EF58322FF
:0A0049000582D5820215831582227C
:10001E00C0E0C0F0C083C082C0D075D00012051001
:0B002E00D0D0D082D083D0F0D0E032E0
:10005600C0E0C0F0C083C082C0D075D000120513C6
:10006600D0D0D082D083D0F0D0E032C0E0C0F0C093
:1000760083C082C0D075D00012058CD0D0D082D07B
:0600860083D0F0D0E0324F
:00000001FF
